:020000040800F2
:1000000000060020A1020008591000081110000885
:10001000391000081110000831100008A302000870
:10002000A3020008A3020008A30200084D2900084B
:10003000A3020008A3020008A3020008A30200080C
:10004000A3020008A3020008A3020008A3020008FC
:10005000A3020008A3020008DD3D0008093E0008D5
:10006000353E0008613E00088D3E0008A3020008EE
:10007000A3020008A3020008A3020008A3020008CC
:10008000A3020008A3020008A3020008A3020008BC
:10009000A3020008A3020008A3020008B93E00085A
:1000A000A3020008A3020008A3020008A30200089C
:1000B000A3020008A3020008A3020008A30200088C
:1000C000A3020008A3020008A3020008A30200087C
:1000D000A3020008A3020008A3020008A30200086C
:1000E0001D3F0008A3020008A3020008A3020008A5
:1000F000A3020008A3020008A3020008A30200084C
:10010000A3020008A3020008A53F0008A3020008FC
:10011000A3020008A3020008A3020008A30200082B
:10012000A3020008A3020008A3020008A30200081B
:10013000A3020008A3020008A3020008A30200080B
:10014000A3020008A3020008A3020008A3020008FB
:10015000A3020008A3020008A3020008A3020008EB
:10016000A3020008A3020008A3020008A3020008DB
:10017000A3020008B9340008A3020008A302000883
:10018000A3020008A3020008913F0008A302000890
:10019000A3020008A3020008A3020008A3020008AB
:1001A000A3020008A3020008A3020008A30200089B
:1001B000A3020008A3020008A3020008A30200088B
:1001C000A3020008A3020008A3020008A30200087B
:1001D000A3020008A5340008A3020008A302000837
:1001E000A3020008A3020008A3020008A30200085B
:1001F000A3020008A3020008A3020008A30200084B
:10020000A3020008A3020008A3020008A30200083A
:10021000A3020008A3020008A3020008A30200082A
:10022000A3020008A3020008A3020008A30200081A
:10023000A3020008A3020008A3020008A30200080A
:10024000A3020008A3020008A3020008A3020008FA
:10025000A3020008A3020008A3020008A3020008EA
:10026000A3020008A3020008A3020008A3020008DA
:10027000A3020008A3020008A3020008A3020008CA
:10028000A3020008A3020008A3020008A3020008BA
:10029000A3020008A3020008A3020008A3020008AA
:1002A00002E000F000F8FEE772B63A4880F30888F2
:1002B000394880F3098839484EF60851CEF20001DA
:1002C000086040F20000CCF200004EF63471CEF22D
:1002D00000010860BFF34F8FBFF36F8F40F2000043
:1002E000C0F2F0004EF68851CEF200010860BFF374
:1002F0004F8FBFF36F8F4FF00000E1EE100A4EF604
:100300003C71CEF200010860062080F31488BFF330
:100310006F8F02F0D9FB02F07BFB03F015FB4FF06F
:1003200055301F491B4A91423CBF41F8040BFAE784
:100330001C49194A91423CBF41F8040BFAE71A499B
:100340001A4A1B4B9A423EBF51F8040B42F8040B69
:10035000F8E700201749184A91423CBF41F8040BC6
:10036000FAE702F093FB03F073FB144C144DAC421C
:1003700003DA54F8041B8847F9E700F041F8114C00
:10038000114DAC4203DA54F8041B8847F9E702F038
:100390007BBB0000000600200022002000000008B7
:1003A0000000002000060020D043000800220020AA
:1003B000642200206822002004470020A0020008D8
:1003C000A0020008A0020008A00200082DE9F04FDA
:1003D0002DED108AC1F80CD0D0F80CD0BDEC108AED
:1003E000BDE8F08F002383F311882846A047002042
:1003F00001F090FEFEE701F00BFE00DFFEE70000DB
:1004000038B502F063FA054602F096FA0446D0B910
:100410000F4B9D4219D001339D4241F2883512BFE6
:10042000044600250124002002F05AFA0CB100F025
:1004300077F800F089FD00F029FC284600F01EF94D
:1004400000F06EF8F9E70025EDE70546EBE700BFA1
:10045000010007B008B500F0E5FBA0F12003584209
:10046000584108BD07B541F21203022101A8ADF8B9
:10047000043000F0F5FB03B05DF804FB38B5202331
:1004800083F311881748C3680BB101F0C9FE00233C
:10049000154A4FF47A71134801F086FE002383F366
:1004A0001188124C236813B12368013B23606368F1
:1004B00013B16368013B63600D4D2B7833B96368FA
:1004C0007BB9022000F0B0FC322363602B78032B51
:1004D00007D163682BB9022000F0A6FC4FF47A73B1
:1004E000636038BD682200207D040008842300205A
:1004F0007C220020084B187003280CD8DFE800F09D
:1005000008050208022000F07FBC022000F06ABC4F
:10051000024B00225A6070477C2200208423002076
:10052000F8B5504B504A1C461968013100F09980CB
:1005300004339342F8D162684C4B9A4240F2918066
:100540004B4B9B6803F1006303F500339A4280F044
:100550008880002000F0B4FB0220FFF7CBFF454B62
:100560000021D3F8E820C3F8E810D3F81021C3F82D
:100570001011D3F81021D3F8EC20C3F8EC10D3F805
:100580001421C3F81411D3F81421D3F8F020C3F8C0
:10059000F010D3F81821C3F81811D3F81821D3F8A4
:1005A000802042F00062C3F88020D3F8802022F03F
:1005B0000062C3F88020D3F88020D3F8802042F076
:1005C0000072C3F88020D3F8802022F00072C3F8B4
:1005D0008020D3F8803072B64FF0E023C3F8084D86
:1005E000D4E90004BFF34F8FBFF36F8F224AC2F8E4
:1005F0008410BFF34F8F536923F480335361BFF3EB
:100600004F8FD2F8803043F6E076C3F3C905C3F3C9
:100610004E335B0103EA060C29464CEA8177013927
:10062000C2F87472F9D2203B13F1200FF2D1BFF35C
:100630004F8FBFF36F8FBFF34F8FBFF36F8F536930
:1006400023F4003353610023C2F85032BFF34F8FBD
:10065000BFF36F8F202383F31188854680F30888CA
:100660002047F8BD0000020820000208FFFF010833
:10067000002200200044025800ED00E02DE9F04F78
:1006800093B0B44B2022FF2100900AA89D6800F08F
:1006900005FCB14A1378A3B90121B0481170C360B9
:1006A000202383F31188C3680BB101F0B9FD002347
:1006B000AB4A4FF47A71A94801F076FD002383F329
:1006C0001188009B13B1A74B009A1A60A64A1378B1
:1006D000032B03D000231370A24A53604FF0000A8B
:1006E000009CD3465646D146012000F08DFB24B134
:1006F0009C4B1B68002B00F02682002000F092FA31
:100700000390039B002BF2DB012000F06BFB039BAB
:10071000213B1F2BE8D801A252F823F09D070008C7
:10072000C507000859080008E9060008E90600089E
:10073000E9060008EB080008BB0A0008D509000814
:10074000370A00085F0A0008850A0008E906000861
:10075000970A0008E9060008090B00083D08000890
:10076000E90600084D0B0008A90700083D0800082D
:10077000E9060008370A0008E9060008E90600084B
:10078000E9060008E9060008E9060008E90600088D
:10079000E9060008E9060008590800080220FFF7EA
:1007A00059FE002840F0F981009B022105A8BAF10A
:1007B000000F08BF1C4641F21233ADF8143000F0B0
:1007C0004FFA91E74FF47A7000F02CFA071EEBDB3A
:1007D0000220FFF73FFE0028E6D0013F052F00F280
:1007E000DE81DFE807F0030A0D101336052304212C
:1007F00005A8059300F034FA17E004215548F9E7FD
:1008000004215A48F6E704215948F3E74FF01C0841
:10081000404608F1040800F055FA0421059005A8A7
:1008200000F01EFAB8F12C0FF2D101204FF00009B0
:1008300000FA07F747EA0B0B5FFA8BFB00F07AFB35
:1008400026B10BF00B030B2B08BF0024FFF70AFEA9
:100850004AE704214748CDE7002EA5D00BF00B0353
:100860000B2BA1D10220FFF7F5FD074600289BD0F6
:100870000120002600F024FA0220FFF73BFE5FFA79
:1008800086F8404600F02CFA0446B0B10399404681
:100890000136A1F140025142514100F031FA0028E5
:1008A000EDD1BA46044641F21213022105A83E4694
:1008B000ADF8143000F0D4F916E725460120FFF713
:1008C00019FE244B9B68AB4207D9284600F0FAF981
:1008D000013040F067810435F3E70025224BBA462A
:1008E0003E461D701F4B5D60A8E7002E3FF45CAFD5
:1008F0000BF00B030B2B7FF457AF0220FFF7FAFD31
:10090000322000F08FF9B0F10008FFF64DAF18F07B
:1009100003077FF449AF0F4A08EB0503926893423F
:100920003FF642AFB8F5807F3FF73EAF124BB84578
:10093000019323DD4FF47A7000F074F90390039A69
:10094000002AFFF631AF039A0137019B03F8012B10
:10095000EDE700BF00220020802300206822002055
:100960007D040008842300207C2200200422002033
:10097000082200200C22002080220020C820FFF73F
:1009800069FD074600283FF40FAF1F2D11D8C5F1B0
:1009900020020AAB25F0030084494245184428BFD1
:1009A0004246019200F054FA019AFF217F4800F07C
:1009B00075FA4FEAA803C8F387027C4928460193D9
:1009C00000F074FA064600283FF46DAF019B05EB7A
:1009D000830533E70220FFF73DFD00283FF4E4AE36
:1009E00000F0ACF900283FF4DFAE0027B846704BAA
:1009F0009B68BB4218D91F2F11D80A9B01330ED018
:100A000027F0030312AA134453F8203C05934046F1
:100A1000042205A9043700F021FB8046E7E73846A9
:100A200000F050F90590F2E7CDF81480042105A8F4
:100A300000F016F902E70023642104A8049300F0F3
:100A400005F900287FF4B0AE0220FFF703FD00286F
:100A50003FF4AAAE049800F067F90590E6E700239A
:100A6000642104A8049300F0F1F800287FF49CAE00
:100A70000220FFF7EFFC00283FF496AE049800F048
:100A800055F9EAE70220FFF7E5FC00283FF48CAEB9
:100A900000F064F9E1E70220FFF7DCFC00283FF4F6
:100AA00083AE05A9142000F05FF9074604210490E5
:100AB00004A800F0D5F83946B9E7322000F0B2F8C2
:100AC000071EFFF671AEBB077FF46EAE384A07EB28
:100AD0000903926893423FF667AE0220FFF7BAFC23
:100AE00000283FF461AE27F003074F44B9453FF4B7
:100AF000A5AE484609F1040900F0E4F80421059088
:100B000005A800F0ADF8F1E74FF47A70FFF7A2FC0A
:100B100000283FF449AE00F011F9002844D00A9BA8
:100B200001330BD008220AA9002000F0BFF90028E9
:100B30003AD02022FF210AA800F0B0F9FFF792FC7A
:100B40001C4801F0EDFA13B0BDE8F08F002E3FF421
:100B50002BAE0BF00B030B2B7FF426AE002364218E
:100B600005A8059300F072F8074600287FF41CAE34
:100B70000220FFF76FFC804600283FF415AEFFF718
:100B800071FC41F2883001F0CBFA059800F01EFAB2
:100B900046463C4600F0CEF9A6E506464EE64FF046
:100BA000000901E6BA467EE637467CE68022002050
:100BB00000220020A08601002DE9F84F4FF47A733F
:100BC00006460D46002402FB03F7DFF85080DFF8ED
:100BD000509098F900305FFA84FA5A1C01D0A34271
:100BE00012D159F824002A4631460368D3F820B0C0
:100BF0003B46D847854207D1074B012083F800A028
:100C0000BDE8F88F0124E4E7002CFBD04FF4FA7024
:100C100001F086FA0020F3E7D02300201022002004
:100C200014220020002307B5024601210DF1070020
:100C30008DF80730FFF7C0FF20B19DF8070003B023
:100C40005DF804FB4FF0FF30F9E700000A4604218D
:100C500008B5FFF7B1FF80F00100C0B2404208BD07
:100C6000074B0A4630B41978064B53F82140014629
:100C700023682046DD69044BAC4630BC604700BFAA
:100C8000D023002014220020A086010070B50A4E57
:100C900000240A4D01F0F2FC30802868338883423A
:100CA00008D901F0E7FC2B6804440133B4F5003F98
:100CB0002B60F2D370BD00BFD22300208C23002014
:100CC00001F0BABD00F1006000F500300068704727
:100CD00000F10060920000F5003001F031BD00002D
:100CE000054B1A68054B1B889B1A834202D9104496
:100CF00001F0C0BC002070478C230020D2230020CC
:100D000038B50446074D29B128682044BDE838406D
:100D100001F0C8BC2868204401F0B2FC0028F3D0E0
:100D200038BD00BF8C2300200020704700F1FF5029
:100D300000F58F10D0F8000870470000064991F8C0
:100D4000243033B100230822086A81F82430FFF7E9
:100D5000BFBF0120704700BF90230020014B1868DF
:100D6000704700BF0010005C1B4B0246F0B51868CE
:100D70001A4BC0F30B06000C1F885C68BE4293F947
:100D8000085003D09F89BE4203D10C335C6893F9AD
:100D900008500426124B1F880433874208BF13F9FA
:100DA000025C013EF7D1013A013C0B460A449342F2
:100DB00007D214F9016F581C2EB1034600F8016CDC
:100DC000F5E7184605E02C2482421C7001D9981CD6
:100DD0005D70401AF0BD00BF0010005C1C220020B6
:100DE00098400008022804D1054B4FF080629A61B8
:100DF00070470128FCD1034B4FF48032F7E700BF66
:100E0000000C025800180258022804D1044B4FF479
:100E100080629A617047012801D1024B9861704746
:100E2000000C025800180258022805D1064A5369DE
:100E300083F48063536170470128FCD1034A5369EE
:100E400083F00103F6E700BF000C025800180258B7
:100E5000002310B5934203D0CC5CC4540133F9E7AE
:100E600010BD0000013810B510F9013F3BB191F9F8
:100E700000409C4203D11AB10131013AF4E71AB1A2
:100E800091F90020981A10BD1046FCE7034602466F
:100E9000D01A12F9011B0029FAD170470244034607
:100EA000934202D003F8011BFAE770472DE9F8439B
:100EB0001F4D14460746884695F8242052BBDFF89C
:100EC00070909CB395F824302BB92022FF2148461E
:100ED0002F62FFF7E3FF95F824004146C0F10802B6
:100EE00005EB8000A24228BF2246D6B29200FFF74F
:100EF000AFFF95F82430A41B17441E449044E4B27D
:100F0000F6B2082E85F82460DBD1FFF717FF002822
:100F1000D7D108E02B6A03EB82038342CFD0FFF7DF
:100F20000DFF0028CBD10020BDE8F8830120FBE7AE
:100F300090230020024B1A78024B1A70704700BFB2
:100F4000D02300201022002038B51A4C1A4D20461C
:100F500000F0E8FB2946204600F010FC2D681748F9
:100F6000D5F89020D2F8043843F00203C2F80438D0
:100F700001F0D6F82846124900F00EFDD5F8902071
:100F8000104DD2F80438286823F002030E49A0421D
:100F9000C2F804384FF4E1330B6001D000F020FBBD
:100FA0006868A04204D00849BDE8384000F018BB8A
:100FB00038BD00BFF8290020AC41000840420F00B6
:100FC000B441000814220020B82300200C4B70B557
:100FD0000C4D04461E780C4B55F826209A420DD035
:100FE0000A4B002118221846FFF758FF04600146FB
:100FF00055F82600BDE8704000F0F2BA70BD00BFA1
:10100000D023002014220020F8290020B82300203B
:1010100000B59BB0EFF3098168226846FFF718FF1F
:10102000EFF30583014B9B6BFEE700BF00ED00E093
:1010300008B5FFF7EDFF000000B59BB0EFF30981A5
:1010400068226846FFF704FFEFF30583014B5B6BF3
:10105000FEE700BF00ED00E0FEE7000030B50A4407
:10106000084D91420DD011F8013B5840082340F340
:101070000004013B2C4013F0FF0384EA5000F6D13A
:10108000EFE730BD2083B8ED02684368114301608B
:1010900003B1184770470000024A136843F0C003C9
:1010A000136070470078004013B50E4C204600F0E6
:1010B0008BFA04F1140000234FF400720A490094E3
:1010C00000F04CF9094B4FF40072094904F1380063
:1010D000009400F0C5F9074A074BC4E9172302B092
:1010E00010BD00BFD4230020402400209910000828
:1010F000402600200078004000E1F505037C30B573
:10110000244C002918BF0C46012B11D1224B9842C8
:101110000ED1224BD3F8E82042F08042C3F8E820F9
:10112000D3F8102142F08042C3F81021D3F81031D7
:101130002268036EC16D03EB52038466B3FBF2F3C6
:101140006268150442BF23F0070503F0070343EA72
:101150004503CB60A36843F040034B60E36843F072
:1011600001038B6042F4967343F001030B604FF070
:10117000FF330B62510505D512F0102205D0B2F1F4
:10118000805F04D080F8643030BD7F23FAE73F23CE
:10119000F8E700BFA8400008D4230020004402580C
:1011A0002DE9F047C66D05463768F46921073462BA
:1011B00019D014F0080118BF8021E20748BF41F0A0
:1011C0002001A3074FF0200348BF41F04001600712
:1011D00048BF41F4807183F31188281DFFF754FF45
:1011E000002383F31188E2050AD5202383F31188B5
:1011F0004FF40071281DFFF747FF002383F3118888
:101200004FF020094FF0000A14F0200838D13B06B7
:1012100016D54FF0200905F1380A200610D589F3BC
:101220001188504600F050F9002836DA0821281DB0
:10123000FFF72AFF27F080033360002383F3118830
:10124000790614D5620612D5202383F31188D5E9D7
:1012500013239A4208D12B6C33B127F04007102199
:10126000281DFFF711FF3760002383F31188E30681
:1012700018D5AA6E1369ABB15069BDE8F04718479D
:1012800089F31188736A284695F86410194000F0B4
:10129000B5F98AF31188F469B6E7B06288F311886A
:1012A000F469BAE7BDE8F087F8B5154682680446E8
:1012B0000B46AA4200D28568A1692669761AB54212
:1012C0000BD218462A46FFF7C3FDA3692B44A3613E
:1012D0002846A3685B1BA360F8BD0CD9AF1B18465A
:1012E0003246FFF7B5FD3A46E1683044FFF7B0FDFE
:1012F000E3683B44EBE718462A46FFF7A9FDE3689D
:10130000E5E7000083689342F7B50446154600D22E
:101310008568D4E90460361AB5420BD22A46FFF735
:1013200097FD63692B4463612846A3685B1BA36038
:1013300003B0F0BD0DD93246AF1B0191FFF788FD18
:1013400001993A46E0683144FFF782FDE3683B4487
:10135000E9E72A46FFF77CFDE368E4E710B50A44B5
:101360000024C361029B8460C16002610362C0E922
:101370000000C0E9051110BD08B5D0E9053293425F
:1013800001D1826882B98268013282605A1C42614E
:1013900019700021D0E904329A4224BFC368436126
:1013A00000F0DAFE002008BD4FF0FF30FBE7000040
:1013B00070B5202304460E4683F31188A568A5B1B5
:1013C000A368A269013BA360531CA361157822693D
:1013D000934224BFE368A361E3690BB120469847B9
:1013E000002383F31188284607E03146204600F0A9
:1013F000A3FE0028E2DA85F3118870BD2DE9F74FCE
:1014000004460E4617469846D0F81C904FF0200A26
:101410008AF311884FF0000B154665B12A46314614
:101420002046FFF741FF034660B94146204600F0E1
:1014300083FE0028F1D0002383F31188781B03B0CA
:10144000BDE8F08FB9F1000F03D001902046C847E6
:10145000019B8BF31188ED1A1E448AF31188DCE797
:10146000C160C361009B82600362C0E90511114441
:10147000C0E9000001617047F8B504460D46164604
:10148000202383F31188A768A7B1A368013BA36059
:1014900063695A1C62611D70D4E904329A4224BF08
:1014A000E3686361E3690BB120469847002080F34D
:1014B000118807E03146204600F03EFE0028E2DABF
:1014C00087F31188F8BD0000D0E9052310B59A42D2
:1014D00001D182687AB982680021013282605A1C87
:1014E00082611C7803699A4224BFC368836100F05B
:1014F00033FE204610BD4FF0FF30FBE72DE9F74FDC
:1015000004460E4617469846D0F81C904FF0200A25
:101510008AF311884FF0000B154665B12A46314613
:101520002046FFF7EFFE034660B94146204600F033
:1015300003FE0028F1D0002383F31188781B03B049
:10154000BDE8F08FB9F1000F03D001902046C847E5
:10155000019B8BF31188ED1A1E448AF31188DCE796
:10156000026843681143016003B1184770470000E7
:101570001430FFF743BF00004FF0FF331430FFF784
:101580003DBF00003830FFF7B9BF00004FF0FF3318
:101590003830FFF7B3BF00001430FFF709BF000079
:1015A0004FF0FF311430FFF703BF00003830FFF772
:1015B00063BF00004FF0FF323830FFF75DBF00001F
:1015C00000207047FFF770BD044B036000234360A9
:1015D000C0E9023301230374704700BFC040000814
:1015E00010B52023044683F31188FFF787FD0223FB
:1015F0002374002383F3118810BD000038B5C3693C
:1016000004460D461BB904210844FFF7A9FF2946EB
:1016100004F11400FFF7B0FE002806DA201D4FF495
:101620008061BDE83840FFF79BBF38BD0268436862
:101630001143016003B118477047000013B5406BB8
:1016400000F58054D4F8A4381A681178042914D10C
:10165000017C022911D11979012312898B4013428F
:101660000BD101A94C3002F06FF8D4F8A44802461F
:10167000019B2179206800F0DFF902B010BD000065
:10168000143001F0F1BF00004FF0FF33143001F0CF
:10169000EBBF00004C3002F0C3B800004FF0FF3346
:1016A0004C3002F0BDB80000143001F0BFBF0000A4
:1016B0004FF0FF31143001F0B9BF00004C3002F0A0
:1016C0008FB800004FF0FF324C3002F089B80000B4
:1016D0000020704710B500F58054D4F8A4381A687B
:1016E0001178042917D1017C022914D159790123D9
:1016F00052898B4013420ED1143001F051FF024643
:1017000048B1D4F8A4484FF4407361792068BDE82B
:10171000104000F07FB910BD406BFFF7DBBF000049
:10172000704700007FB5124B012504260446036074
:101730000023057400F1840243602946C0E90233A6
:101740000C4B0290143001934FF44073009601F05B
:1017500003FF094B04F69442294604F14C0002941D
:10176000CDE900634FF4407301F0CAFF04B070BDCF
:10177000E8400008191700083D1600080A682023F1
:1017800083F311880B790B3342F823004B79133321
:1017900042F823008B7913B10B3342F8230000F594
:1017A0008053C3F8A41802230374002383F3118821
:1017B0007047000038B5037F044613B190F85430E9
:1017C000ABB90125201D0221FFF730FF04F1140001
:1017D0006FF00101257700F0CBFC04F14C0084F898
:1017E00054506FF00101BDE8384000F0C1BC38BD75
:1017F00010B5012104460430FFF718FF00232377BA
:1018000084F8543010BD000038B50446002514306B
:1018100001F0BAFE04F14C00257701F089FF201D8C
:1018200084F854500121FFF701FF2046BDE83840FD
:10183000FFF750BF90F8803003F06003202B06D1F3
:1018400090F881200023212A03D81F2A06D80020DF
:101850007047222AFBD1C0E91D3303E0034A4267E7
:1018600007228267C3670120704700BF342200202F
:1018700037B500F58055D5F8A4381A6811780429D1
:101880001AD1017C022917D11979012312898B40C1
:10189000134211D100F14C04204602F009F858B16E
:1018A00001A9204601F050FFD5F8A4480246019B4B
:1018B0002179206800F0C0F803B030BD01F10B03BE
:1018C000F0B550F8236085B004460D46FEB12023E4
:1018D00083F3118804EB8507301D0821FFF7A6FE6E
:1018E000FB6806F14C005B691B681BB1019001F0BD
:1018F00039FF019803A901F027FF024648B1039B75
:101900002946204600F098F8002383F3118805B09B
:10191000F0BDFB685A691268002AF5D01B8A013BAA
:101920001340F1D104F18002EAE70000133138B529
:1019300050F82140ECB1202383F3118804F5805343
:10194000D3F8A4281368527903EB8203DB689B6900
:101950005D6845B104216018FFF768FE294604F16F
:10196000140001F027FE2046FFF7B4FE002383F3A6
:10197000118838BD7047000001F01AB901234022D8
:10198000002110B5044600F8303BFFF787FA00232A
:10199000C4E9013310BD000010B52023044683F3D1
:1019A00011882422416000210C30FFF777FA20468D
:1019B00001F020F902232370002383F3118810BD66
:1019C00070B500EB8103054650690E461446DA6097
:1019D00018B110220021FFF761FAA06918B1102296
:1019E0000021FFF75BFA31462846BDE8704001F060
:1019F00013BA000083682022002103F0011310B500
:101A0000044683601030FFF749FA2046BDE81040D5
:101A100001F08EBAF0B4012500EB810447898D40B6
:101A2000E4683D43A469458123600023A2606360AC
:101A3000F0BC01F0ABBA0000F0B4012500EB81046A
:101A400007898D40E4683D43646905812360002374
:101A5000A2606360F0BC01F021BB000070B50223FE
:101A600000250446242203702946C0F888500C3013
:101A700040F8045CFFF712FA204684F8705001F039
:101A80005FF963681B6823B129462046BDE87040B2
:101A9000184770BD037880F88C30052303704368C5
:101AA0001B6810B504460BB1042198470023A360BE
:101AB00010BD000090F88C20436802701B680BB1C9
:101AC000052118477047000070B590F87030044643
:101AD00013B1002380F8703004F18002204601F039
:101AE0004BFA63689B68B3B994F8803013F06005D3
:101AF00035D00021204601F0F5FC0021204601F000
:101B0000E5FC63681B6813B106212046984706234D
:101B100084F8703070BD204698470028E4D0B4F8AF
:101B20008630A26F9A4288BFA36794F98030A56F70
:101B3000002B4FF0200380F20381002D00F0F28093
:101B4000092284F8702083F3118800212046D4E90B
:101B50001D23FFF771FF002383F31188DAE794F860
:101B6000812003F07F0343EA022340F202329342D2
:101B700000F0C58021D8B3F5807F48D00DD8012B67
:101B80003FD0022B00F09380002BB2D104F18802E9
:101B900062670222A267E367C1E7B3F5817F00F0C5
:101BA0009B80B3F5407FA4D194F88230012BA0D163
:101BB000B4F8883043F0020332E0B3F5006F4DD043
:101BC00017D8B3F5A06F31D0A3F5C063012B90D81F
:101BD0006368204694F882205E6894F88310B4F815
:101BE0008430B047002884D0436863670368A367E4
:101BF0001AE0B3F5106F36D040F6024293427FF4FC
:101C000078AF5C4B63670223A3670023C3E794F8B4
:101C10008230012B7FF46DAFB4F8883023F00203DB
:101C2000A4F88830C4E91D55E56778E7B4F880303A
:101C3000B3F5A06F0ED194F88230204684F88A3034
:101C400001F0DCF863681B6813B101212046984756
:101C5000032323700023C4E91D339CE704F18B03A5
:101C600063670123C3E72378042B10D1202383F378
:101C700011882046FFF7BEFE85F3118803216368B3
:101C800084F88B5021701B680BB12046984794F85C
:101C90008230002BDED084F88B30042323706368FD
:101CA0001B68002BD6D0022120469847D2E794F833
:101CB000843020461D0603F00F010AD501F04EF9CD
:101CC000012804D002287FF414AF2B4B9AE72B4B4A
:101CD00098E701F035F9F3E794F88230002B7FF4B0
:101CE00008AF94F8843013F00F01B3D01A062046E1
:101CF00002D501F00FFCADE701F000FCAAE794F873
:101D00008230002B7FF4F5AE94F8843013F00F018D
:101D1000A0D01B06204602D501F0E4FB9AE701F0B3
:101D2000D5FB97E7142284F8702083F311882B46A3
:101D30002A4629462046FFF76DFE85F31188E9E61D
:101D40005DB1152284F8702083F3118800212046AC
:101D5000D4E91D23FFF75EFEFDE60B2284F8702018
:101D600083F311882B462A4629462046FFF764FE56
:101D7000E3E700BF184100081041000814410008C3
:101D800038B590F870300446002B3ED0063BDAB2EE
:101D90000F2A34D80F2B32D8DFE803F0373131085F
:101DA000223231313131313131313737856FB0F84D
:101DB00086309D4214D2C3681B8AB5FBF3F203FB45
:101DC00012556DB9202383F311882B462A462946E4
:101DD000FFF732FE85F311880A2384F870300EE095
:101DE000142384F87030202383F3118800232046C5
:101DF0001A461946FFF70EFE002383F3118838BDFB
:101E0000C36F03B198470023E7E70021204601F0A4
:101E100069FB0021204601F059FB63681B6813B180
:101E20000621204698470623D7E7000010B590F812
:101E300070300446142B29D017D8062B05D001D8B2
:101E40001BB110BD093B022BFBD80021204601F03D
:101E500049FB0021204601F039FB63681B6813B180
:101E6000062120469847062319E0152BE9D10B23BC
:101E700080F87030202383F3118800231A46194616
:101E8000FFF7DAFD002383F31188DAE7C3689B6963
:101E90005B68002BD5D1C36F03B19847002384F84A
:101EA0007030CEE7024B0022C3E900339A607047DE
:101EB00040280020002382680374054B1B68996842
:101EC0009142FBD25A6803604260106058607047CC
:101ED0004028002008B5202383F31188037C032BBE
:101EE00005D0042B0DD02BB983F3118808BD4369AD
:101EF00000221A604FF0FF334361FFF7DBFF00233E
:101F0000F2E7D0E9003213605A60F3E700238268F9
:101F10000374054B1B6899689142FBD85A680360AB
:101F2000426010605860704740280020054B1969D6
:101F300008741868026853601A60186101230374FA
:101F4000FEF744BA402800204B1C30B5044687B049
:101F50000A4D10D02B6901A8094A00F025F9204646
:101F6000FFF7E4FF049B13B101A800F059F92B69B6
:101F7000586907B030BDFFF7D9FFF8E740280020C7
:101F8000D51E000838B50C4D044641612B698168A7
:101F90009A68914203D8BDE83840FFF78BBF1846D6
:101FA000FFF7B4FF01232C61014623742046BDE8EE
:101FB0003840FEF70BBA00BF40280020044B1A68D7
:101FC0001B6990689B68984294BF0020012070476D
:101FD0004028002010B5084C236820691A68546016
:101FE0002260012223611A74FFF790FF01462069E5
:101FF000BDE81040FEF7EAB94028002008B5FFF719
:10200000DDFF18B1BDE80840FFF7E4BF08BD0000E0
:10201000FFF7E0BFFEE7000010B50C4CFFF742FFF2
:1020200000F0B4F880220A49204600F03BF8012372
:1020300044F8180C037400F099FC002383F3118812
:1020400062B60448BDE8104000F04CB86828002093
:102050001C4100082C41000800F01CB9EFF311806E
:1020600020B9EFF30583202282F311887047000026
:1020700010B530B9EFF30584C4F3080414B180F34C
:10208000118810BDFFF7BAFF84F31188F9E700004B
:10209000034A516853685B1A9842FBD8704700BFE7
:1020A000001000E082600222028270478368A3F180
:1020B0007C0243F80C2C026943F83C2C426943F83B
:1020C000382C074A43F81C2CC268A3F1180043F8C7
:1020D000102C022203F8082C002203F8072C70476A
:1020E000E503000810B5202383F31188FFF7DEFF16
:1020F00000210446FFF746FF002383F311882046A2
:1021000010BD0000024B1B6958610F20FFF70EBF86
:1021100040280020202383F31188FFF7F3BF00003D
:1021200008B50146202383F311880820FFF70CFF30
:10213000002383F3118808BD49B1064B42681B692F
:1021400018605A60136043600420FFF7FDBE4FF033
:10215000FF307047402800200368984206D01A6874
:102160000260506018465961FFF7A4BE7047000036
:1021700038B504460D462068844200D138BD036856
:1021800023605C604561FFF795FEF4E7054B4FF077
:10219000FF3103F11402C3E905220022C3E907124B
:1021A000704700BF4028002070B51C4E05460C4605
:1021B000C0E9032301F0B2FB334653F8142F9A42CF
:1021C0000DD130620A2C2CBF00190A302A60C5E9F3
:1021D0000124C6E90555BDE8704001F089BB316AAC
:1021E000431AE31838BF1C469368A34202D9081962
:1021F00001F08EFB73699A6894420CD85A68AC60FF
:102200002B606A6015609A685D60121B9A604FF0DF
:10221000FF33F36170BDA41A1B68ECE7402800206F
:1022200038B51B4C636998420DD08168D0E9003203
:1022300013605A600022C2609A680A449A604FF0A4
:10224000FF33E36138BD03682246002142F8143FA2
:1022500093425A60C16003D1BDE8384001F052BBDF
:102260009A688168256A0A449A6001F057FB63699D
:10227000411B9A688A42E5D9AB181D1A206A092DBC
:1022800098BF01F10A02BDE83840104401F040BB9C
:10229000402800202DE9F041184C002704F11406D5
:1022A000656901F03BFB236AAA68C11A8A4215D806
:1022B0001344D5F80C802362D5E9003213605A60CC
:1022C0006369EF60B34201D101F01CFB87F3118811
:1022D0002869C047202383F31188E1E76169B1428F
:1022E00009D013441B1ABDE8F0410A2B2CBFC018BB
:1022F0000A3001F00DBBBDE8F08100BF402800208E
:1023000000207047FEE70000704700004FF0FF30EC
:102310007047000002290CD0032904D00129074886
:1023200018BF00207047032A05D8054800EBC200FB
:102330007047044870470020704700BF10420008F3
:1023400044220020C441000870B59AB005460846F2
:10235000144601A900F0C2F801A8FEF797FD431C3E
:102360000022C6B25B001046C5E900342370032387
:10237000023404F8013C01ABD1B202348E4201D8E0
:102380001AB070BD13F8011B013204F8010C04F8F7
:10239000021CF1E708B5202383F311880348FFF7F7
:1023A00067FA002383F3118808BD00BFF8290020D5
:1023B00090F8803003F01F02012A07D190F88120A5
:1023C0000B2A03D10023C0E91D3315E003F060039D
:1023D000202B08D1B0F884302BB990F88120212A25
:1023E00003D81F2A04D8FFF725BA222AEBD0FAE730
:1023F000034A426707228267C3670120704700BF14
:102400003B22002007B5052917D8DFE801F019168F
:1024100003191920202383F31188104A0121019008
:10242000FFF7CEFA019802210D4AFFF7C9FA0D48CD
:10243000FFF7EAF9002383F3118803B05DF804FB8A
:10244000202383F311880748FFF7B4F9F2E720232C
:1024500083F311880348FFF7CBF9EBE764410008E9
:1024600088410008F829002038B50C4D0C4C2A464C
:102470000C4904F10800FFF767FF05F1CA0204F1F7
:1024800010000949FFF760FF05F5CA7204F1180052
:102490000649BDE83840FFF757BF00BFD0420020D3
:1024A00044220020444100084E41000859410008E0
:1024B00070B5044608460D46FEF7E8FCC6B2204655
:1024C000013403780BB9184670BD32462946FEF731
:1024D000C9FC0028F3D10120F6E700002DE9F04700
:1024E00005460C46FEF7D2FC2C49C6B22846FFF73B
:1024F000DFFF08B10836F6B229492846FFF7D8FFB2
:1025000008B11036F6B2632E0BD8DFF89080DFF8F2
:102510009090244FDFF898A02E7846B92670BDE839
:10252000F08729462046BDE8F04701F09FBD252EE3
:1025300030D1072241462846FEF794FC80B91A4B59
:10254000224603F10C0153F8040B8B4242F8040BB2
:10255000F9D1198807359B780F3411809370DBE728
:10256000082249462846FEF77DFC98B9A21C0F4B6D
:10257000197802320909C95D02F8041C13F8011B1D
:1025800001F00F015345C95D02F8031CF0D1183466
:102590000835C1E7013504F8016BBDE7304200089A
:1025A00059410008484200083842000800E8F11F7D
:1025B0000CE8F11FBFF34F8F044B1A695107FCD190
:1025C000D3F810215207F8D1704700BF0020005205
:1025D00008B50D4B1B78ABB9FFF7ECFF0B4BDA6876
:1025E000D10704D50A4A5A6002F188325A60D3F8FA
:1025F0000C21D20706D5064AC3F8042102F188321D
:10260000C3F8042108BD00BF2E4500200020005261
:102610002301674508B5114B1B78F3B9104B1A69B4
:10262000510703D5DA6842F04002DA60D3F810218E
:10263000520705D5D3F80C2142F04002C3F80C2113
:10264000FFF7B8FF064BDA6842F00102DA60D3F810
:102650000C2142F00102C3F80C2108BD2E450020D8
:10266000002000520F289ABF00F58060400400202F
:10267000704700004FF40030704700001020704792
:102680000F2808B50BD8FFF7EDFF00F500330268FF
:10269000013204D104308342F9D1012008BD002069
:1026A000FCE700000F2870B5054645D8FFF7D6FCBB
:1026B000224CFFF77FFF0646FFF78AFF4FF0FF33FC
:1026C000072D6361C4F8143120D82361FFF772FF2E
:1026D0002B0243F02403E360E36843F08003E360EC
:1026E00023695A07FCD42846FFF764FF4FF40031F2
:1026F000FFF7B8FF00F002F93046FFF78BFFFFF756
:10270000B7FC2846BDE87040FFF7BABFC4F81031E7
:10271000FFF750FFA5F108031B0243F02403C4F8A0
:102720000C31D4F80C3143F08003C4F80C31D4F8E8
:1027300010315B07FBD4D6E7002070BD00200052AB
:102740002DE9F84F40EA020305460C461746D80625
:1027500002D00020BDE8F88F27F01F07DFF8D4B0C3
:10276000FFF736FF2744BC4203D10120FFF752FF99
:10277000F0E720222946204601F068FC10B92035F8
:102780002034F0E72B4605F120021E68711CE0D1D1
:1027900004339A42F9D1FFF761FC05F17843234AEB
:1027A000B3F5801F224B28BF9A4603F1040338BFBC
:1027B0009046A2F1080228BF9846A3F108033ABF49
:1027C0009146DA469946FFF7F5FEC8F80060A5EB9A
:1027D000040CD9F8002004F11C0142F00202C9F8EF
:1027E0000020221FDAF8006016F00506FAD152F830
:1027F000043F8A424CF80230F4D1BFF34F8FFFF709
:10280000D9FE4FF0FF32C8F80020D9F8002022F09E
:102810000202C9F80020FFF72BFC2022214628469F
:1028200001F014FC0028AAD030469FE71420005283
:10283000102100521020005210B5084C237828B106
:102840001BB9FFF7C5FE0123237010BD002BFCD080
:102850002070BDE81040FFF7DDBE00BF2E45002010
:102860000244074BD2B210B5904200D110BD441CB7
:1028700000B253F8200041F8040BE0B2F4E700BFC7
:10288000504000580E4B30B51C6F240405D41C6F0B
:102890001C671C6F44F400441C670A4C0244236804
:1028A000D2B243F480732360074B904200D130BD15
:1028B000441C51F8045B00B243F82050E0B2F4E746
:1028C00000440258004802585040005807B5012201
:1028D00001A90020FFF7C4FF019803B05DF804FBD5
:1028E00013B50446FFF7F2FFA04205D0012201A96B
:1028F00000200194FFF7C6FF02B010BD0144BFF3F2
:102900004F8F064B884204D3BFF34F8FBFF36F8FB7
:102910007047C3F85C022030F4E700BF00ED00E030
:10292000034B1A681AB9034AD2F8D0241A607047C8
:10293000304500200040025808B5FFF7F1FF024B78
:102940001868C0F3806008BD30450020EFF30983AC
:10295000054968334A6B22F001024A6383F3098810
:10296000002383F31188704700EF00E0202080F3FC
:10297000118862B60D4B0E4AD96821F4E061090452
:10298000090C0A430B49DA60D3F8FC2042F080724C
:10299000C3F8FC20084AC2F8B01F116841F00101D9
:1029A00011601022DA7783F82200704700ED00E012
:1029B0000003FA0555CEACC5001000E0202310B589
:1029C00083F311880E4B5B6813F4006314D0F1EEAF
:1029D000103AEFF309844FF08073683CE361094BD0
:1029E000DB6B236684F30988FFF7E8FA10B1064B26
:1029F000A36110BD054BFBE783F31188F9E700BF26
:102A000000ED00E000EF00E0F7030008FA03000823
:102A100070B5BFF34F8FBFF36F8F1A4A0021C2F812
:102A20005012BFF34F8FBFF36F8F536943F40033DE
:102A30005361BFF34F8FBFF36F8FC2F88410BFF3A2
:102A40004F8FD2F8803043F6E074C3F3C900C3F36C
:102A50004E335B0103EA0406014646EA81750139FB
:102A6000C2F86052F9D2203B13F1200FF2D1BFF32C
:102A70004F8F536943F480335361BFF34F8FBFF3DC
:102A80006F8F70BD00ED00E0FEE700000A4B0B48C1
:102A90000B4A90420BD30B4BC11EDA1C121A22F0C8
:102AA00003028B4238BF00220021FEF7F7B953F82A
:102AB000041B40F8041BECE73444000804470020E2
:102AC00004470020044700207047000070B5D0E99B
:102AD000244300224FF0FF359E6804EB421351015E
:102AE000D3F80009002805DAD3F8000940F0804047
:102AF000C3F80009D3F8000B002805DAD3F8000B5F
:102B000040F08040C3F8000B013263189642C3F8CE
:102B10000859C3F8085BE0D24FF00113C4F81C3821
:102B200070BD000000EB8103D3F80CC02DE9F04329
:102B3000DCF814204E1CD0F89050D2F800E005EBE1
:102B4000063605EB4118506870450AD30122D5F8C6
:102B5000343802FA01F123EA0101C5F83418BDE85E
:102B6000F083AEEB0003BCF81040A34228BF23461D
:102B7000D8F81849A4B2B3EB840FF0D89468A4F144
:102B8000040959F8047F3760A4EB09071F44042F98
:102B9000F7D81C44034494605360D4E7890141F0A2
:102BA0002001016103699B06FCD41220FFF770BA73
:102BB00010B50A4C2046FEF7E1FE094BC4F89030F0
:102BC000084BC4F89430084C2046FEF7D7FE074B5C
:102BD000C4F89030064BC4F8943010BD3445002042
:102BE0000000084080420008D0450020000004405A
:102BF0008C42000870B503780546012B5DD1494B26
:102C0000D0F89040984259D1474B0E216520D3F817
:102C1000D82042F00062C3F8D820D3F8002142F057
:102C20000062C3F80021D3F80021D3F8802042F0DD
:102C30000062C3F88020D3F8802022F00062C3F83D
:102C40008020D3F8803000F071FC384BE360384BC3
:102C5000C4F800380023D5F89060C4F8003EC023C3
:102C600023604FF40413A3633369002BFCDA0123C0
:102C70000C203361FFF70CFA3369DB07FCD4122018
:102C8000FFF706FA3369002BFCDA00262846A66017
:102C9000FFF71CFF6B68C4F81068DB68C4F81468A1
:102CA000C4F81C68002B3AD1224BA3614FF0FF33CC
:102CB0006361A36843F00103A36070BD1E4B98429B
:102CC000C8D1194B0E214D20D3F8D82042F0007204
:102CD000C3F8D820D3F8002142F00072C3F80021D5
:102CE000D3F80021D3F8802042F00072C3F880208E
:102CF000D3F8802022F00072C3F88020D3F880201F
:102D0000D3F8D82022F08062C3F8D820D3F800216D
:102D100022F08062C3F80021D3F8003193E7074B1B
:102D2000C3E700BF3445002000440258401400406F
:102D300003002002003C30C0D0450020083C30C0D9
:102D4000F8B5D0F89040054600214FF000662046C7
:102D5000FFF724FFD5F8941000234FF001128F687D
:102D60004FF0FF30C4F83438C4F81C2804EB431289
:102D700001339F42C2F80069C2F8006BC2F808092B
:102D8000C2F8080BF2D20B68D5F89020C5F898303D
:102D9000636210231361166916F01006FBD112202E
:102DA000FFF776F9D4F8003823F4FE63C4F800384E
:102DB000A36943F4402343F01003A3610923C4F83B
:102DC0001038C4F814380B4BEB604FF0C043C4F814
:102DD000103B094BC4F8003BC4F81069C4F8003933
:102DE000D5F8983003F1100243F48013C5F8982009
:102DF000A362F8BD5C42000840800010D0F890202B
:102E000090F88A10D2F8003823F4FE6343EA0113E5
:102E1000C2F80038704700002DE9F84300EB810349
:102E2000D0F890500C468046DA680FFA81F94801D4
:102E3000166806F00306731E022B05EB41134FF0D4
:102E4000000194BFB604384EC3F8101B4FF00101C7
:102E500004F1100398BF06F1805601FA03F391695B
:102E600098BF06F5004600293AD0578A04F1580168
:102E7000374349016F50D5F81C180B430021C5F8A2
:102E80001C382B180127C3F81019A7405369611E7D
:102E90009BB3138A928B9B08012A88BF5343D8F8AF
:102EA0009820981842EA034301F140022146C8F8ED
:102EB0009800284605EB82025360FFF76FFE08EB8F
:102EC0008900C3681B8A43EA845348341E43640163
:102ED0002E51D5F81C381F43C5F81C78BDE8F8837F
:102EE00005EB4917D7F8001B21F40041C7F8001B78
:102EF000D5F81C1821EA0303C0E704F13F030B4A8D
:102F00002846214605EB83035A60FFF747FE05EB91
:102F10004910D0F8003923F40043C0F80039D5F83F
:102F20001C3823EA0707D7E70080001000040002DE
:102F3000D0F894201268C0F89820FFF7C7BD0000B1
:102F40005831D0F8903049015B5813F4004004D058
:102F500013F4001F0CBF0220012070474831D0F845
:102F6000903049015B5813F4004004D013F4001F63
:102F70000CBF02200120704700EB8101CB68196A69
:102F80000B6813604B6853607047000000EB8103CF
:102F900030B5DD68AA691368D36019B9402B84BFC6
:102FA000402313606B8A1468D0F890201C4402EB15
:102FB0004110013C09B2B4FBF3F46343033323F043
:102FC000030343EAC44343F0C043C0F8103B2B68FB
:102FD00003F00303012B0ED1D2F8083802EB4110A5
:102FE00013F4807FD0F8003B14BF43F0805343F0CC
:102FF0000053C0F8003B02EB4112D2F8003B43F013
:103000000443C2F8003B30BD2DE9F041D0F8906098
:1030100005460C4606EB4113D3F8087B3A07C3F884
:10302000087B08D5D6F814381B0704D500EB8103BC
:10303000DB685B689847FA071FD5D6F81438DB07BA
:103040001BD505EB8403D968CCB98B69488A5A68CB
:10305000B2FBF0F600FB16228AB91868DA689042D3
:103060000DD2121AC3E90024202383F311882146CC
:103070002846FFF78BFF84F31188BDE8F081012318
:1030800003FA04F26B8923EA02036B81CB68002BFD
:10309000F3D021462846BDE8F041184700EB8103F4
:1030A0004A0170B5DD68D0F890306C692668E6603A
:1030B00056BB1A444FF40020C2F810092A6802F0E7
:1030C0000302012A0AB20ED1D3F8080803EB421416
:1030D00010F4807FD4F8000914BF40F0805040F015
:1030E0000050C4F8000903EB4212D2F8000940F086
:1030F0000440C2F800090122D3F8340802FA01F1B1
:103100000143C3F8341870BD19B9402E84BF402064
:10311000206020681A442E8A8419013CB4FBF6F41E
:1031200040EAC44040F00050C6E700002DE9F041FD
:10313000D0F8906004460D4606EB4113D3F80879A9
:10314000C3F80879FB071CD5D6F81038DA0718D56C
:1031500000EB8103D3F80CC0DCF81430D3F800E0A6
:10316000DA6896451BD2A2EB0E024FF000081A60F7
:10317000C3F80480202383F31188FFF78FFF88F3BF
:1031800011883B0618D50123D6F83428AB401342EA
:1031900012D029462046BDE8F041FFF7C3BC012309
:1031A00003FA01F2038923EA02030381DCF8083001
:1031B000002BE6D09847E4E7BDE8F0812DE9F84F11
:1031C000D0F8905004466E69AB691E4016F48058E2
:1031D0006E6103D0BDE8F84FFEF740BC002E12DA56
:1031E000D5F8003E9F0705D0D5F8003E23F0030335
:1031F000C5F8003ED5F80438204623F00103C5F891
:103200000438FEF757FC300505D52046FFF75EFC75
:103210002046FEF73FFCB1040CD5D5F8083813F072
:10322000060FEB6823F470530CBF43F4105343F4C0
:10323000A053EB60320704D56368DB680BB120460E
:103240009847F30200F1BA80B70226D5D4F89090DF
:1032500000274FF0010A09EB4712D2F8003B03F4B4
:103260004023B3F5802F11D1D2F8003B002B0DDAAB
:1032700062890AFA07F322EA0303638104EB8703F6
:10328000DB68DB6813B13946204698470137D4F82C
:103290009430FFB29B689F42DDD9F00619D5D4F86F
:1032A0009000026AC2F30A1702F00F0302F4F01250
:1032B000B2F5802F00F0CC80B2F5402F09D104EB9D
:1032C0008303002200F58050DB681B6A974240F0C0
:1032D000B2803003D5F8185835D5E90303D500215D
:1032E0002046FFF791FEAA0303D501212046FFF7F0
:1032F0008BFE6B0303D502212046FFF785FE2F03CB
:1033000003D503212046FFF77FFEE80203D5042101
:103310002046FFF779FEA90203D505212046FFF7D5
:1033200073FE6A0203D506212046FFF76DFE2B02CD
:1033300003D507212046FFF767FEEF0103D50821DB
:103340002046FFF761FE700340F1A980E90703D52D
:1033500000212046FFF7EAFEAA0703D501212046F7
:10336000FFF7E4FE6B0703D502212046FFF7DEFEE0
:103370002F0703D503212046FFF7D8FEEE0603D51D
:1033800004212046FFF7D2FEA80603D505212046DA
:10339000FFF7CCFE690603D506212046FFF7C6FEDF
:1033A0002A0603D507212046FFF7C0FEEB0576D598
:1033B00020460821BDE8F84FFFF7B8BED4F890903A
:1033C00000274FF0010AD4F894305FFA87FB9B681E
:1033D0009B453FF639AF09EB4B13D3F8002902F4B4
:1033E0004022B2F5802F24D1D3F80029002A20DA18
:1033F000D3F8002942F09042C3F80029D3F80029FD
:10340000002AFBDB5946D4F89000FFF7C7FB22895E
:103410000AFA0BF322EA0303238104EB8B03DB6834
:103420009B6813B159462046984759462046FFF7F6
:1034300079FB0137C7E7910701D1D0F80080072A4F
:1034400002F101029CBF03F8018B4FEA18283DE707
:1034500004EB830300F58050DA68D2F818C0DCF87A
:103460000820DCE9001CA1EB0C0C00218F4208D1E4
:10347000DB689B699A683A449A605A683A445A6091
:1034800027E711F0030F01D1D0F800808C4501F13E
:10349000010184BF02F8018B4FEA1828E6E7BDE876
:1034A000F88F000008B50348FFF788FEBDE8084024
:1034B000FFF784BA3445002008B50348FFF77EFEC5
:1034C000BDE80840FFF77ABAD0450020D0F8903028
:1034D00003EB4111D1F8003B43F40013C1F8003B6A
:1034E00070470000D0F8903003EB4111D1F800395B
:1034F00043F40013C1F8003970470000D0F8903051
:1035000003EB4111D1F8003B23F40013C1F8003B59
:1035100070470000D0F8903003EB4111D1F800392A
:1035200023F40013C1F8003970470000090100F1CD
:103530006043012203F56143C9B283F8001300F030
:103540001F039A4043099B0003F1604303F5614365
:10355000C3F880211A60704730B50433039C0172B0
:10356000002104FB0325C160C0E90653049B0363EB
:10357000059BC0E90000C0E90422C0E90842C0E997
:103580000A11436330BD00000022416AC260C0E9F5
:103590000411C0E90A226FF00101FEF7E9BD000045
:1035A000D0E90432934201D1C2680AB9181D7047AC
:1035B00000207047036919600021C2680132C260AF
:1035C000C269134482699342036124BF436A036161
:1035D000FEF7C2BD38B504460D46E3683BB16269EB
:1035E0000020131D1268A3621344E36207E0237AEC
:1035F00033B929462046FEF79FFD0028EDDA38BD95
:103600006FF00100FBE70000C368C269013BC360C3
:103610004369134482699342436124BF436A43610F
:1036200000238362036B03B11847704770B52023F2
:10363000044683F31188866A3EB9FFF7CBFF05463F
:1036400018B186F31188284670BDA36AE26A13F8A0
:10365000015B9342A36202D32046FFF7D5FF00230C
:1036600083F31188EFE700002DE9F84F04460E467A
:10367000174698464FF0200989F311880025AA467D
:10368000D4F828B0BBF1000F09D141462046FFF71E
:10369000A1FF20B18BF311882846BDE8F88FD4E94B
:1036A0000A12A7EB050B521A934528BF9346BBF1AC
:1036B000400F1BD9334601F1400251F8040B9142EF
:1036C00043F8040BF9D1A36A403640354033A36276
:1036D000D4E90A239A4202D32046FFF795FF8AF3E2
:1036E0001188BD42D8D289F31188C9E730465A46BD
:1036F000FDF7AEFBA36A5E445D445B44A362E7E76B
:1037000010B5029C0433017204FB0321C460C0E9BC
:1037100006130023C0E90A33039B0363049BC0E93B
:103720000000C0E90422C0E90842436310BD000064
:10373000026A6FF00101C260426AC0E904220022FD
:10374000C0E90A22FEF714BDD0E904239A4201D150
:10375000C26822B9184650F8043B0B60704700203D
:1037600070470000C3680021C2690133C360436928
:10377000134482699342436124BF436A4361FEF765
:10378000EBBC000038B504460D46E3683BB1236945
:1037900000201A1DA262E2691344E36207E0237A63
:1037A00033B929462046FEF7C7FC0028EDDA38BDBC
:1037B0006FF00100FBE7000003691960C268013A7D
:1037C000C260C269134482699342036124BF436AA1
:1037D000036100238362036B03B118477047000045
:1037E00070B520230D460446114683F31188866A7E
:1037F0002EB9FFF7C7FF10B186F3118870BDA36A19
:103800001D70A36AE26A01339342A36204D3E169A3
:1038100020460439FFF7D0FF002080F31188EDE740
:103820002DE9F84F04460D46904699464FF0200A80
:103830008AF311880026B346A76A4FB94946204645
:10384000FFF7A0FF20B187F311883046BDE8F88F5D
:10385000D4E90A073A1AA8EB0607974228BF174689
:10386000402F1BD905F1400355F8042B9D4240F829
:10387000042BF9D1A36A40364033A362D4E90A236A
:103880009A4204D3E16920460439FFF795FF8BF390
:1038900011884645D9D28AF31188CDE729463A46A0
:1038A000FDF7D6FAA36A3D443E443B44A362E5E7F4
:1038B000D0E904239A4217D1C3689BB1836A8BB1C4
:1038C000043B9B1A0ED01360C368013BC360C369FD
:1038D0001A4483699A42026124BF436A0361002348
:1038E00083620123184670470023FBE700F0DAB833
:1038F000034B002258631A610222DA60704700BF4E
:10390000000C0040014B0022DA607047000C0040C0
:10391000014B5863704700BF000C0040014B586AD0
:10392000704700BF000C00404B6843608B688360A9
:10393000CB68C3600B6943614B6903628B69436267
:103940000B6803607047000008B53C4B40F2FF7104
:103950003B48D3F888200A43C3F88820D3F888204E
:1039600022F4FF6222F00702C3F88820D3F88820EF
:10397000D3F8E0200A43C3F8E020D3F808210A4333
:10398000C3F808212F4AD3F808311146FFF7CCFFBE
:1039900000F5806002F11C01FFF7C6FF00F58060B2
:1039A00002F13801FFF7C0FF00F5806002F1540119
:1039B000FFF7BAFF00F5806002F17001FFF7B4FF76
:1039C00000F5806002F18C01FFF7AEFF00F580602A
:1039D00002F1A801FFF7A8FF00F5806002F1C40121
:1039E000FFF7A2FF00F5806002F1E001FFF79CFF06
:1039F00000F5806002F1FC01FFF796FF02F58C7183
:103A000000F58060FFF790FF00F004F90E4BD3F84B
:103A1000902242F00102C3F89022D3F8942242F09F
:103A20000102C3F894220522C3F898204FF0605297
:103A3000C3F89C20054AC3F8A02008BD00440258E2
:103A4000000002589842000800ED00E01F00080343
:103A500008B500F0DBFAFEF7DFFA0F4BD3F8DC20F5
:103A600042F04002C3F8DC20D3F8042122F04002E7
:103A7000C3F80421D3F80431084B1A6842F0080255
:103A80001A601A6842F004021A60FEF749FFBDE8A6
:103A90000840FEF7E9BC00BF004402580018024885
:103AA00070470000114BD3F8E82042F00802C3F839
:103AB000E820D3F8102142F00802C3F810210C4A84
:103AC000D3F81031D36B43F00803D363C722094BFB
:103AD0009A624FF0FF32DA6200229A615A63DA602A
:103AE0005A6001225A611A60704700BF00440258B0
:103AF0000010005C000C0040094A08B51169D36849
:103B00000B40D9B29B076FEA0101116107D5202351
:103B100083F31188FEF7A0FA002383F3118808BD10
:103B2000000C00403A4B4FF0FF31D3F8802062F098
:103B30000042C3F88020D3F8802002F00042C3F88E
:103B40008020D3F88020D3F88420C3F88410D3F8E1
:103B500084200022C3F88420D3F88400D86F40F07A
:103B6000FF4040F4FF0040F43F5040F03F00D86772
:103B7000D86F20F0FF4020F4FF0020F43F5020F0E9
:103B80003F00D867D86FD3F888006FEA40506FEADB
:103B90005050C3F88800D3F88800C0F30A00C3F877
:103BA0008800D3F88800D3F89000C3F89010D3F8B9
:103BB0009000C3F89020D3F89000D3F89400C3F895
:103BC0009410D3F89400C3F89420D3F89400D3F859
:103BD0009800C3F89810D3F89800C3F89820D3F849
:103BE0009800D3F88C00C3F88C10D3F88C00C3F87D
:103BF0008C20D3F88C00D3F89C00C3F89C10D3F829
:103C00009C10C3F89C20D3F89C3000F0D3B900BFBF
:103C100000440258614B0122C3F80821604BD3F8DD
:103C2000F42042F00202C3F8F420D3F81C2142F041
:103C30000202C3F81C210222D3F81C31594BDA606E
:103C40005A689104FCD5584A1A6001229A60574A72
:103C5000DA6000221A614FF440429A61514B9A692E
:103C60009204FCD51A6842F480721A604C4B1A6FA9
:103C700012F4407F04D04FF480321A6700221A6792
:103C80001A6842F001021A60454B1A685007FCD5C9
:103C900000221A611A6912F03802FBD10121196061
:103CA0004FF0804159605A67414ADA62414A1A61CD
:103CB0001A6842F480321A60394B1A689103FCD5B5
:103CC0001A6842F480521A601A689204FCD53A4A83
:103CD0003A499A6200225A6319633949DA6399634F
:103CE0005A64384A1A64384ADA621A6842F0A852AA
:103CF0001A602B4B1A6802F02852B2F1285FF9D1F2
:103D000048229A614FF48862DA6140221A622F4A8F
:103D1000DA644FF080521A652D4A5A652D4A9A6529
:103D200032232D4A1360136803F00F03022BFAD1DC
:103D30001B4B1A6942F003021A611A6902F0380239
:103D4000182AFAD1D3F8DC2042F00052C3F8DC2064
:103D5000D3F8042142F00052C3F80421D3F804211F
:103D6000D3F8DC2042F08042C3F8DC20D3F80421F1
:103D700042F08042C3F80421D3F80421D3F8DC20B8
:103D800042F00042C3F8DC20D3F8042142F00042A4
:103D9000C3F80421D3F80431704700BF00800051FC
:103DA000004402580048025800C000F00200000120
:103DB0000000FF01008890082220400063020901F2
:103DC0002C02040047040508FD0BFF012000002021
:103DD0000010E00000010100002000524FF0B0424E
:103DE00008B5D2F8883003F00103C2F8883023B157
:103DF000044A13680BB150689847BDE80840FEF7C5
:103E0000DDBD00BF844600204FF0B04208B5D2F8B7
:103E1000883003F00203C2F8883023B1044A936863
:103E20000BB1D0689847BDE80840FEF7C7BD00BF9A
:103E3000844600204FF0B04208B5D2F8883003F035
:103E40000403C2F8883023B1044A13690BB15069E6
:103E50009847BDE80840FEF7B1BD00BF844600208A
:103E60004FF0B04208B5D2F8883003F00803C2F82A
:103E7000883023B1044A93690BB1D0699847BDE8F3
:103E80000840FEF79BBD00BF844600204FF0B042C3
:103E900008B5D2F8883003F01003C2F8883023B197
:103EA000044A136A0BB1506A9847BDE80840FEF710
:103EB00085BD00BF844600204FF0B04310B5D3F855
:103EC000884004F47872C3F88820A30604D5124A07
:103ED000936A0BB1D06A9847600604D50E4A136BFB
:103EE0000BB1506B9847210604D50B4A936B0BB16D
:103EF000D06B9847E20504D5074A136C0BB1506CA0
:103F00009847A30504D5044A936C0BB1D06C98472D
:103F1000BDE81040FEF752BD844600204FF0B0438C
:103F200010B5D3F8884004F47C42C3F888206205B9
:103F300004D5164A136D0BB1506D9847230504D56F
:103F4000124A936D0BB1D06D9847E00404D50F4A27
:103F5000136E0BB1506E9847A10404D50B4A936EB3
:103F60000BB1D06E9847620404D5084A136F0BB1A9
:103F7000506F9847230404D5044A936F0BB1D06F58
:103F80009847BDE81040FEF719BD00BF84460020E9
:103F900008B50348FDF704F9BDE80840FEF70EBD7B
:103FA000D423002008B5FFF7A7FDBDE80840FEF7C1
:103FB00005BD0000062108B50846FFF7B7FA06213F
:103FC0000720FFF7B3FA06210820FFF7AFFA062112
:103FD0000920FFF7ABFA06210A20FFF7A7FA06210E
:103FE0001720FFF7A3FA06212820FFF79FFA0921DF
:103FF0007A20FFF79BFA07213220FFF797FA0C216E
:104000005220BDE80840FFF791BA000008B5FFF75D
:1040100089FD00F00DF8FDF7D5FAFDF7ADFCFDF7D1
:104020007FFBFFF73DFDBDE80840FFF75FBC0000E8
:104030000023054A19460133102BC2E9001102F191
:104040000802F8D1704700BF8446002010B501393E
:104050000244904201D1002005E0037811F8014F9D
:10406000A34201D0181B10BD0130F2E7034611F83E
:10407000012B03F8012B002AF9D1704753544D331B
:104080003248373F3F3F0053544D33324837343383
:104090002F3735330000000001105A00031059007B
:1040A0000120580003205600009600000000000088
:1040B0000000000000000000000000000000000000
:1040C000000000008D15000879150008B5150008DE
:1040D000A1150008AD150008991500088515000800
:1040E00071150008C1150008000000009D160008A9
:1040F00089160008C5160008B1160008BD1600088C
:10410000A91600089516000881160008D1160008A7
:104110000000000001000000000000006D61696EF9
:104120000000000069646C65000000002441000884
:1041300080280020F8290020010000001520000838
:10414000000000004172647550696C6F7400254274
:104150004F415244252D424C002553455249414C74
:10416000250000000200000000000000BD1800084B
:104170002D19000840004000A0420020B04200205D
:10418000020000000000000003000000000000002A
:10419000751900080000000010000000C042002057
:1041A0000000000001000000000000003445002075
:1041B000010102000524000815230008B1230008AE
:1041C0009523000843000000CC4100080902430089
:1041D000020100C0320904000001020201000524AE
:1041E0000010010524010001042402020524060038
:1041F00001070582030800FF09040100020A00000C
:104200000007050102400000070581024000000090
:1042100012000000184200081201100102000040C4
:1042200009124157000201020301000004030904BE
:1042300025424F4152442500594A5541565F413667
:1042400053455F48373433003031323334353637F5
:104250003839414243444546000000000000000058
:10426000C91A0008811D00082D1E000840004000EA
:104270006C4600206C460020010000007C460020B7
:104280008000000040010000080000000001000064
:1042900000040000080000000100802A0000000067
:1042A000AAAAAAAA01000024FFFF00000000000043
:1042B00000A00A000000000000000000AAAAAAAAAC
:1042C00000000000FFFF00000000000000000000F0
:1042D0000000004000000000AAAAAAAA00000040B6
:1042E000FFFF0000000000000000000000001000C0
:1042F00000040000AAAAAAAA00000000FFFF000014
:104300000000000000000000408516400080000012
:10431000AAAAAAAA40451500FFFF000000000070ED
:10432000070000000000000000000000AAAAAAAADE
:1043300000000000FFFF000000000000000000007F
:104340000100000001000000AAAAAAAA00000000C3
:10435000FFFF00000000000000000000000000005F
:1043600000000000AAAAAAAA00000000FFFF0000A7
:10437000000000000000000000000000000000003D
:10438000AAAAAAAA00000000FFFF00000000000087
:10439000000000000000000000000000AAAAAAAA75
:1043A00000000000FFFF000000000000000000000F
:1043B0000000000000000000AAAAAAAA0000000055
:1043C000FFFF0000000000000000000000000000EF
:1043D000750400000000000000001E000000000046
:1043E000FF000000F8290020D42300200000000076
:1043F0007C4000083F000000500400008740000897
:104400003F00000000960000000008009600000039
:1044100000080000040000002C420008000000001A
:10442000000000000000000000000000000000008C
:044430000000000088
:00000001FF
